:020000040000FA
:0400000004303A2866
:08000800A000030EA100831209
:100010008B1C32288B1031181428B11C3228643004
:10002000010203183128182800001628172818285C
:1000300019281A281B281C281D281E281F283110A3
:10004000B114A810031005190314AA0DA90DA80DC9
:10005000B00B322831152A08AF002908AE00280855
:10006000AD00B11081010B11210E8300A00E200EF6
:02007000090085
:0C007400203084008001840A6030040207
:10008000031C3C281230B00092218316FF239000FD
:10009000831283160C308505870183128501870141
:1000A000073099000030831691009F008312C830FA
:1000B00083168100831231309000003083168C004B
:1000C000831210308B00831600309B001C141A081A
:1000D0008312BC00831610309B001C141A08831274
:1000E000BD00EE21831620309B001C141A088312D9
:1000F000C2000130C21BC200C2080319C200810144
:100100008E018F010B118B100B108C018B17962019
:100110003119AC20B30B9428031085190314B90DC1
:10012000F030390203191521EF21872864003118B6
:1001300008000B1D08000B11B11031141230B00073
:10014000051DA728321483160113831208003210EC
:10015000831601178312080031110130B7008B1389
:100160002030370783169B001C141A088312A40042
:10017000A500C030A5061030370783169B001C145D
:100180001A088312A3000030370783169B001C1443
:100190001A088312A2008B17321CD42822090339B3
:1001A000A200A309A409A50922082D02031D0F29F5
:1001B00023082E02031D0F2924082F02031DF528F2
:1001C00001303702031DE7283D143E14932102300D
:1001D0003702031DEE28BD143E149F210330370261
:1001E000031DF5283D153E14AB2125082F02031DE4
:1001F0000F2901303702031D00293D103E14BC2198
:1002000002303702031D0729BD103E14BD21033003
:100210003702031D0E293D113E14BE210F29B70AD6
:100220000430370203180800AF280130B600B300CD
:10023000B400B500B70085018701B113DD21962018
:10024000B30B4229031085190314B90DF03039029C
:1002500003196929B41F8501B41F8701B40B422912
:10026000B50B42290230B500013037020319C42111
:10027000023037020319C921033037020319D32191
:10028000FA30B400311D1F293111321C4C292D09BF
:100290000339AD00AE09AF092F1CB1132F1C1F2964
:1002A000B11B1F292E181F29B1178B1320303707B8
:1002B000BB002F08BA007F2110303707BB002E0883
:1002C000BA007F2100303707BB002D08BA007F211C
:1002D0008B17E02185018701B70AB6010430370288
:1002E000031C1F29C0010800EE2108003E1C080065
:1002F0003E101030BB003D08BA007F2108008B1370
:100300003A0883161C159A003B089B0055309D0047
:10031000AA309D009C1464009C188B291C11831228
:100320008B17080008008516051285100510C001FE
:10033000C0148E018F010C104208C1000800851600
:10034000051285100510C00140158E018F010C109B
:100350004208C10008008512051285140510C0016D
:10036000C0158E018F010C104208C1000800080062
:10037000080008000800080008000800080008003D
:100380000800080008000800380903398500B80093
:100390000800C00A38093339B800C01C0339C01836
:1003A000303985000800380930398500B800080068
:1003B00008000800080008000800B801B814080088
:1003C000B80101303702031DE729B814381602308E
:1003D0003702031DED290000B816080008000C1CA8
:1003E00087280C10C10B87284208C1008501C0185E
:1003F000051440198514C0190516C0018E018F011E
:080400000C104208C1000800C5
:084000000300030003000800A7
:02400E00CC01E3
:10420000010003000300030003000200020002009B
:1042100002000000000000000000FF00FF00FF009F
:10422000000000000000000000000000000000008E
:104230000000C000C000C000C000FF00FF00FF0081
:104240000100C300F300CF00FF00C300F300CF0064
:10425000FF00C300F300CF00FF00FF00FF00FF00DE
:10426000FF00FF00FF00FF00FF00FF00FF00FF0056
:10427000FF00FF00FF00FF00FF00FF00FF00FF0046
:10428000FF00FF00FF00FF00FF00FF00FF00FF0036
:10429000FF00FF00FF00FF00FF00FF00FF00FF0026
:1042A000FF00FF00FF00FF00FF00FF00FF00FF0016
:1042B000FF00FF00FF00FF00FF00FF00FF00FF0006
:1042C000FF00FF00FF00FF00FF00FF00FF00FF00F6
:1042D000FF00FF00FF00FF00FF00FF00FF00FF00E6
:1042E000FF00FF00FF00FF00FF00FF00FF00FF00D6
:1042F000FF00FF00FF00FF00FF00FF00FF00AA001B
:00000001FF
